:0300000002006D8E
:200033003753656D656E74746573742056657273696F6E20312E302020766F6D2030392E4C
:2000530030392E323030312C20496E7465726E657420446F776E6C6F6164758170D2B7D285
:20007300B6D2B5D2B47550007551017552027553039000D57DFF7C147B2FDD10DC0E055043
:200093000551055205537C14DB0280D911A380EAE55093F590C2B711D0E55193D2B7F590E6
:2000B300C2B611D0E55293D2B6F590C2B511D0E55393D2B5F590C2B411D0D2B4227E2FDE44
:2000D300FE2281B7C292B49888B38090A08CC986C8E801374212341808330010200C490601
:1200F3004868FFCEA4ACEF97CDAE8EE0EE858FFEDF7F61
:00010501F9
